:1000000010308A0000280000A100030E8301A20026
:100010000A08A3008A010C1C0F28A60A0C100B1D4D
:1000200025280B111530A400A40B142800003D3026
:100030008100A503031D3628000000000000000019
:1000400010100130A0008B1236280B1C2C2806083B
:100050000230A0000B1036280C1D3628241C332833
:100060002418071134280715A4090C1123088A0045
:10007000220E8300A10E210E09000A108A100A1117
:10008000820770346E3475346D340A108A100A1188
:1000900082076E3475346D3420340A108A100A11C8
:1000A000820728340C34013406340A108A100A11ED
:1000B00082070C3400340A108A100A118207203497
:1000C0002034433461346C346934623472346134C2
:1000D000743469346F346E3400340A108A100A1193
:1000E00082073034203420346E34483400340A100F
:1000F0008A100A118207203443346F346E346E3410
:1001000065346334743420344C347834203400340F
:100110000A108A100A11820730342E3430343034F9
:10012000203420347034463400340A108A100A1106
:100130008207203420344534723472346F34723480
:10014000203443347834203400340A108A100A11E1
:10015000820730342E343034203410341134433498
:1001600000340A108A100A118207203420344334E4
:100170006F346E346E3465346334743420347434C4
:1001800065346D34703400340A108A100A11820705
:1001900020342034313430347534733420342834EE
:1001A000353430344B3448347A34293400340A102E
:1001B0008A100A11820720342034323430347534E6
:1001C000733420342834323435344B3448347A3460
:1001D000293400340A108A100A118207203420348E
:1001E0003534303475347334203428343134303479
:1001F0004B3448347A34293400340A148A100A11F2
:100200008207203420343134303430347534733440
:100210002034283435344B3448347A34293400348B
:100220000A148A100A1182072034323430343034F0
:10023000753473342034283432342E3435344B340E
:1002400048347A34293400340A148A100A11820797
:100250002034203435343034303475347334203421
:10026000283431344B3448347A34293400340A1475
:100270008A100A1182072034203431346D347334EB
:1002800020342034283435343034303448347A340F
:10029000293400340A148A100A11820720342034C9
:1002A00032346D34733420342034283432343534CD
:1002B000303448347A34293400340A148A100A114C
:1002C00082072034203435346D34733420342034A4
:1002D000283431343034303448347A3429340034DA
:1002E0000A148A100A118207203420343134303441
:1002F0006D34733420342034283435343034483469
:100300007A34293400340A148A100A1182072034FE
:100310002034323430346D34733420342034283473
:100320003234353448347A34293400340A148A108B
:100330000A11820720342034353430346D3473345C
:100340002034203428343134303448347A34293459
:1003500000340A148A100A118207203420343534FC
:10036000303430346D347334203420342834313414
:1003700048347A34293400340A148A100A11820766
:1003800020342034353475347334203428343134F7
:10039000303430344B3448347A34293400340A143D
:1003A0008A100A11820704340A3411341F3480344D
:1003B00000340A148A100A11820720345634653436
:1003C0007234733469346F346E34203431342E34E3
:1003D0003034313400340A148A100A118207283468
:1003E0006334293420344F344B3431345834473457
:1003F0004C342034323430343034343400340A1045
:100400008A140A1182074D344F344434453443343E
:1004100078344E3455344C344C3400340A108A1439
:100420000A1182074D344F34443445344C34783407
:100430004E3455344C344C3400340A108A140A11AA
:1004400082074D344F3444344534203420342B3427
:1004500054344D345034203420344E3455344C34DC
:100460004C3400340A108A140A1182074D344F3478
:1004700044344534203420342B3450344C345A34F2
:1004800020345734493444345434483400346C30C4
:100490008400000803195D2A0130F800BF30F7001E
:1004A0006400F70B502AF80B4E2A4A30F700F70B7E
:1004B000572A00006400800B4C2A00340508C33919
:1004C000F300720DF700F70DFC30F70577083C39A3
:1004D000730485008514831685100000831285102F
:1004E0008316851083120034F008031D792A051045
:1004F0007A2A051483160510F10E7108F200831292
:100500005E22F10E7108F2005E220D30F700F70B4B
:10051000872A00341430EC004722C3308316850547
:10052000831205108316051083128510831685101B
:100530008312B6013608023C031CA62A0230EC00E6
:1005400047220330F2005E22B60A9A2A0D30F700E5
:10055000F70BA82A0230F2005E220D30F700F70BED
:10056000AF2AB6013608023C031CC22A36084D20C9
:10057000B700F0013708F10074220230EC00472286
:10058000B60AB22A8A110A1640280130F00038084B
:10059000F10074220034871707170A30EC00472255
:1005A00087130713003401306C02EE006D08023C23
:1005B000031DDC2A4030EE076E088038EF00F001A2
:1005C0006F08F100742200346B08F7000C307702DA
:1005D0000319F72A0A3077020319FF2A0D30770230
:1005E0000319052B0830770203190A2B0F2BF00192
:1005F0000130F10074220230EC0047221B2B013045
:10060000EC000230ED00D3221B2B0130EC00ED009A
:10061000D3221B2BF0011030F10074221B2B6B082E
:100620001F3C031C152B0730EB050130F0006B0855
:10063000F10074221B2B0034B630F700FA01F901E7
:10064000F8015A085B045C045D04031D292BF701C3
:10065000362B0310F81B352BDA0DDB0DDC0DDD0D11
:10066000FA0DF90DF80DF70B292BF8138A110A1260
:10067000DD2B5D080319AA2BE50061080319AA2BDD
:10068000E507031C442B4B2B7F30E502031CAA2BF0
:100690000319AA2B4F2B8130E5070318AA2B6508F5
:1006A000F700F801F901FA015E08E900E9175F08AF
:1006B000E8006008E7001830E500E601671C782BC9
:1006C0006408FA07031C6A2BF90A031D6A2BF80A4F
:1006D0000319E6176308F907031C712BF80A0319BD
:1006E000E6176208DF00DF175F08F8070318E61750
:1006F000E60DF80CF90CFA0CE90CE80CE70C031009
:10070000E50B5D2B0130F7070318AA2BF81B8F2B85
:10071000E90DFA0DF90DF80DF7030319AA2BE91FDE
:10072000A02BFA0A031DA02BF90A031DA02BF80A1F
:10073000031DA02BF80CF90CFA0CF70A0319AA2BCD
:100740005E08E6006208E606E61FA82BF817AE2B47
:10075000F813AE2BF701F801F901FA01000000349B
:1007600010108E018F01A6010030A00010143D3042
:1007700081000530A5000B118B16A008031DC12BAD
:10078000BD2B0F08FA000E08F7000F087A02031DB0
:10079000C12B7708D9007A08DA00FA012608F90097
:1007A0005908F7005A08F8007A08DD007908DC00DB
:1007B0007808DB007708DA001C2BE001DF01DE019E
:1007C0008130DD007A08E4007908E3007808E2006F
:1007D0007708E10039237A08D8007908D70078082B
:1007E000D6007708D5005808E0005708DF00560803
:1007F000DE005508DD005808E4005708E3005608FD
:10080000E2005508E10039230034871787160A30C3
:10081000EC00472287138712003480300318DE066D
:10082000E3015A08E2005E08E20659080319FA2CAF
:10083000E100F7005D080319032DE1020319A02C64
:100840000318232C5F2C5E08E700E7175F08E6001B
:100850006008E500E4010310E70CE60CE50CE40C8D
:10086000E10B2A2CE21F372C6314172D6310611043
:1008700063165C3084002D2D6312E21B492C611C31
:10088000542CE70CE60CE50CE40CF70A0319122DC6
:10089000542CE71B572C0310E40DE50DE60DE70D76
:1008A000F7030319122D492C6317BF2C63135A0841
:1008B000E200DA1F5D2CE7170B2DE7130B2D5D0807
:1008C000E100F7005908E1025A08E700E7175B0862
:1008D000E6005C08E500E4010310E70CE60CE50C1B
:1008E000E40CE10B6B2CE21F782CE314172DE310C2
:1008F0006110E316603084002D2DE312E21B8A2C78
:10090000611C952CE70CE60CE50CE40CF70A0319C6
:10091000122D952CE71B982C0310E40DE50DE60D28
:10092000E70DF7030319122D8A2CE317BF2CE313ED
:100930005E08E200DE1F9E2CE7170B2DE7130B2D40
:100940005E08E700E7175F08E6006008E500E21FC1
:10095000AD2CE7136315172D6311E40161105C30B2
:1009600084002D2DE21BD52C5A08E200611CBF2CFF
:10097000E70CE60CE50CE40CF70A0319122DE41F52
:10098000D02CE50A031DD02CE60A031DD02CE70A63
:10099000031DD02CE70CE60CE50CF70A0319122D09
:1009A000631B562CE31B972CF42C8030E706E71FC3
:1009B000DD2C172D5E08E200EA2C5A08E200E70859
:1009C000031DEA2CE608031DEA2CE508031DEA2CAA
:1009D000F7010B2DE71BF42C0310E40DE50DE60DDC
:1009E000E70DF70BEA2C122DE21FF82CE7170B2D61
:1009F000E7130B2D5D08F7005E08E7005F08E600CF
:100A00006008E5000B2D5908F7005A08E7005B085D
:100A1000E6005C08E5006708F8006608F90065086C
:100A2000FA004C2DF701F801F901FA014C2DE4010F
:100A3000E509E609E709E409E40A031D262DE50AAC
:100A4000031D262DE60A031D262DE70A6318362C02
:100A5000E318772C6319AC2CDA2C0008E507031C8B
:100A6000372DE60A031D372DE70A031961148403A5
:100A70000008E607031C3F2DE70A031961148403ED
:100A80000008801B442D803AE70703186114631A9D
:100A90003C2CE31A7D2CB22C0000003458080319BA
:100AA000142EE4005C080319142EE4020318592DD7
:100AB0005E2D7F30E4070318142E642D8130E4028C
:100AC000031C142E0319142E6408F700F801F90111
:100AD000FA01E3015908E200E2175A08E1005B0855
:100AE000E0001930E4005F08E0020318872D0130B0
:100AF000E1020318872DE2020318872DE302031891
:100B0000872DE30AE20AE10A5F08E007B92D5E08D3
:100B1000E1020318A22D0130E2020318A22DE30224
:100B20000318A22DE30AE20A5E08E1075F08E00766
:100B3000031CB92DE10A031DB92DE20A031DB92DCD
:100B4000E30AB92D5D088038E2020318B82D0130A0
:100B5000E3020318B82DE30A5D088038E2075E0857
:100B6000E107031C962DE20A031D962DE30A962D3C
:100B70007A14E40BBC2DC72D0310E00DE10DE20D3E
:100B8000E30D0310FA0DF90DF80DE50D732D651C3D
:100B9000CF2D0310F80CF90CFA0CE50CD22DF7034D
:100BA0000319142EE51BFB2D0310E00DE10DE20DE2
:100BB000E30D5F08E0020318E72D0130E10203189E
:100BC000E72DE2020318E72DE302031C0A2E5E085C
:100BD000E1020318F22D0130E2020318F22DE302C4
:100BE000031C0A2E5D088038E2020318FB2D013039
:100BF000E302031C0A2EFA0A031D0A2EF90A031D3A
:100C00000A2EF80A031D0A2EF70A0319142EF80CEF
:100C1000F90CFA0C5908E4005D08E406E41F122EF2
:100C2000F817182EF813182EF701F801F901FA0138
:100C3000000000340130EC00ED00D322D50155084E
:100C40000F3C031C282E2030EB00E422D50A1F2E77
:100C50000130EC00ED00D3220034861F312E061B3C
:100C6000352E1430EC0047222D2EA00100345F08F1
:100C7000E6006308E606E61F422E03110310DF1BA1
:100C80000314752E5F08E6006208E7005E08E702BD
:100C90000319502EE61F752E0308013A8300752EA6
:100CA0006308E7005F08E70203195C2EE61F752E54
:100CB0000308013A8300752E6408E7006008E70224
:100CC0000319682EE61F752E0308013A8300752E5E
:100CD0006508E7006108E7020319742EE61F752E08
:100CE0000308013A8300752E031000340130D90047
:100CF0005508F7005608F8005708F9005808FA0098
:100D0000F8137708DA007808DB007908DC007A0845
:100D1000DD00E101E0012030DF008230DE005D080F
:100D2000E5005C08E4005B08E3005A08E2003726AF
:100D3000031CB52E5808E0005708DF005608DE00F7
:100D40005508DD00CD30E400CC30E3004C30E2004B
:100D50007B30E10039237A08D8007908D700780879
:100D6000D6007708D500D90A782E5908F800003443
:100D7000071607170A30EC004722071207138A11DB
:100D80000A16DE2C8316061083120610A630F70012
:100D9000F70BC82E000083160614061483120618DB
:100DA000D42E0030F800EF2E1530F700F70BD62EBA
:100DB0000000831606148312061CE02E5010E12E4C
:100DC00050144F30F700F70BE32E00000000501CCA
:100DD000ED2E0130F800EF2EEF2E0030F800003439
:100DE000D1015108073C031C1E2F831606108312E5
:100DF00006100330F700F70BFB2E0310D00C031C7A
:100E00000B2F831606140000831206180A2F0030D9
:100E1000F800202F142F8316061083120610061CCC
:100E2000142F0030F800202F1030F700F70B162F8A
:100E30000000831606148312D10AF12E0130F80047
:100E400000348E30F7005508F8005408F900FA0114
:100E5000F808031D352F7908F800F9010830F7026A
:100E6000F808031D352FF7013D2F0310F81B3C2F09
:0E0E7000F90DF80DF703352FF81300000034CC
:101000000408DF00E001D71F0A282D30EB008A1109
:10101000E4228A15D71756080319AE287F305602E6
:10102000031C6928D600E5010430E6000310D90D41
:10103000D80DD70DE00DE60B162804305602031824
:10104000292803305602031DA3280A306002031C1E
:10105000A3280330D602E50A50210310D90DD80D7C
:10106000D70DE00D39210230E6000310E00CD70C5B
:10107000D80CD90CE60B352850210430E6000310BB
:10108000E10CE20CE30CE40CE60B3F283921502183
:101090006308E4006208E3006108E200E10139212D
:1010A00050216208E4006108E300E101E201392116
:1010B000E0191D28D608031D6228D90AD80AD70AC4
:1010C000E00AA3280310D90DD80DD70DE00DD603E3
:1010D0001D28D609D60A7F30D607E5010430E60080
:1010E0000310D90DD80DD70DE00DE60B7028043094
:1010F000D60705305602031CB02850210310D90D25
:10110000D80DD70DE00D0310D90DD80DD70DE00D7A
:1011100039210310D90DD80DD70DE00DE50A0330A4
:10112000E6000310E00CD70CD80CD90CE60B912884
:101130000330D602601E79280310E00CD70CD80CBF
:10114000D90CD6037928D609D60A0330D607650804
:10115000DB006508DD005F0ADD07DD285F0AE500CA
:101160003030EB008A11E4228A15DF080319372991
:101170002E30EB008A11E4228A156508DE00DE03BA
:101180005F085E02031CC6285F08DE00DE08031944
:10119000D0283030EB008A11E4228A15DE0BC928F2
:1011A0006508E6005F0AE60203185929D6035F0ABC
:1011B000DD006508DD025D08DB006008DA00560826
:1011C0000319E728DC000310DA0CDC0BE3285D08C8
:1011D0000319372930305A07EB008A11E4228A15A7
:1011E0005B08031DFB28DF08031937292E30EB00AD
:1011F0008A11E4228A15DB03DD0303193729560817
:1012000003190729DC000310DA0DDC0B03295A0847
:10121000E0026008E1005708E2005808E3005908BE
:10122000E4000310D90DD80DD70DE00D0310D90D32
:10123000D80DD70DE00D6408D907031C2429D80F59
:101240002429D70F2429E00A6308D807031C2B2977
:10125000D70F2B29E00A6208D7070318E00A6108B4
:10126000E0070310D90DD80DD70DE00DDD280000E3
:1012700059296408D907031C4229D80F4229D70FDE
:101280004229E00A6308D807031C4929D70F4929D6
:10129000E00A6208D7070318E00A6108E007003493
:1012A0006008E1005708E2005808E3005908E4002C
:1012B0000034000000340130C1004310CB01CA01EA
:1012C000C901C8012008023C031D9429061B6C2992
:1012D00083160614402B8312861B94294708CB00E3
:1012E0004608CA004508C9004408C8004314013034
:1012F000C1008A111A268A150630EC000130ED0073
:101300008A11D3228A15D00150088A11A5208A1586
:10131000D00AEB008A11E4228A1507305002031D1F
:1013200084298A112D268A154108FD3E03183B2B7E
:10133000033E442BC20B9E290230C1003B2B8A1175
:10134000C2268A15F808031DBC298A111A268A1597
:10135000D00150088A11B1208A15D00AEB008A11F9
:10136000E4228A150E305002031DA929CB01CA01BF
:10137000C901C80143100A2BCC30D0008A11F026D5
:101380008A15BE30D0008A11F0268A15C0014008A7
:10139000083C031CFA2936304007D000D101D101A6
:1013A0005108073C031CF22983160610831206100D
:1013B0000430F700F70BDA2900008316061400004A
:1013C0000000000000000000061483120618EA293D
:1013D0000310EB290314D20C2130F700F70BEE2990
:1013E000D10AD0295208F8005008840078088000FB
:1013F000C00AC7293630D0000930D100D501D60146
:10140000510856020318192A56085007840000088C
:10141000D3000830D20053085506D400D40C550828
:101420000318183AD500D50CD30CD20B0B2AD60AC8
:10143000002AD5080319202A0030F800222A222A7F
:101440000130F800F80803190A2B0310B60C371CFA
:101450002A2AB6173708FA003608D4003708D5000C
:101460008A1121278A157A08C7007908C6007808EA
:10147000C5007708C40003144708DC004608DB00F9
:101480004508DA004408D900E001DF01DE017D30C3
:10149000DD008A110D248A157708D0007808D10064
:1014A0007908D2007A08D300D5013C08D4008A110B
:1014B00021278A150314DC01DB01DA018330D9000E
:1014C0007A08E0007908DF007808DE007708DD00A0
:1014D0008A110D248A157708D4007808D500790878
:1014E000D6007A08D700DB005608DA005508D90084
:1014F0005408D800DF01DE01DD018330DC008A11F1
:101500004E258A1503105308DC005208DB005108F1
:10151000DA005008D9007A08E0007908DF0078087E
:10152000DE007708DD008A110D248A157A08C700CD
:101530007908C6007808C5007708C4000314470876
:10154000DC004608DB004508DA004408D9004B08F7
:10155000E0004A08DF004908DE004808DD008A1183
:101560000D248A157A08CF007908CE007808CD00BE
:101570007708CC008A111A268A154F08D8004E0821
:10158000D7004D08D6004C08D5008A1176268A155A
:101590007808063CD000EC000130ED008A11D3221F
:1015A0008A15E101E001DF01DE014F08E5004E0888
:1015B000E4004D08E3004C08E2008A1137268A1542
:1015C0000318E42A031DE92A2030EB008A11E422E3
:1015D0008A15013084004F08D9004E08D8004D0804
:1015E000D7004C08D60000202030EB008A11E422FE
:1015F0008A15431C002B1030EB008A11E4228A1557
:101600001130EB008A11E4228A154330EB008A1175
:10161000E4228A150130C1008A11C2268A15F80811
:10162000031D292B8A111A268A15D00150088A1108
:10163000B1208A15D00AEB008A11E4228A150E30F7
:101640005002031D162BCB01CA01C901C80143106A
:101650003A2BCC30D0008A11F0268A154430D000C5
:101660008A11F0268A158316061083120614043098
:10167000C200C1013B2B8A11B0238A15622983164F
:1016800083128A110A160B2F0A148A140A11820770
:101690009A290C2B9F29271127088316870083126C
:1016A0000715A40183160108C039203881000930CC
:1016B000831203178D008F0183168C130C14831271
:1016C0000C080313B6008A111A268A153608F23E52
:1016D0000318CF2C0E3E182DB70137088A11C420ED
:1016E0008A15B70AEB008A11E4228A150E303702F8
:1016F000031D6D2B0030F800043892001330831660
:101700009200831207110C30970096010A30950061
:10171000CF2CB70137088A11D7208A15B70AEB00FA
:101720008A11E4228A150E303702031D8A2B0030FD
:10173000F8000438920027308316920083120711B4
:101740000C309700960114309500CF2CB701370864
:101750008A11EA208A15B70AEB008A11E4228A1559
:101760000E303702031DA72B0030F800043892001A
:10177000633083169200831207110C309700960194
:1017800032309500CF2CB70137088A11FD208A1519
:10179000B70AEB008A11E4228A150E303702031DC6
:1017A000C42B0030F80004389200C7308316920032
:1017B000831207110C309700960164309500CF2CEE
:1017C000B70137088A1110218A15B70AEB008A1170
:1017D000E4228A150F303702031DE12B0030F80098
:1017E00005389200633083169200831207110C3083
:1017F0009700960132309500CF2CB70137088A1137
:1018000024218A15B70AEB008A11E4228A150E30CA
:101810003702031DFE2B0030F80005389200F93026
:1018200083169200831207110C30970096017D30C9
:101830009500CF2C0030F800920000308316920003
:101840008312B70137088A1137218A15B70AEB00CE
:101850008A11E4228A150E303702031D222C0B3028
:1018600097008530900003309600E830950083168D
:101870000C158312CF2CB70137088A114A218A151B
:10188000B70AEB008A11E4228A150E303702031DD5
:101890003C2C07309600D0309500CF2CB70137088C
:1018A0008A115D218A15B70AEB008A11E4228A1594
:1018B0000E303702031D4F2C1330960088309500F0
:1018C000CF2CB70137088A1170218A15B70AEB00AF
:1018D0008A11E4228A150E303702031D622C27304C
:1018E000960010309500CF2CB70137088A1183215C
:1018F0008A15B70AEB008A11E4228A150E303702E6
:10190000031D752C4E30960020309500CF2CB7016A
:1019100037088A1196218A15B70AEB008A11E4224A
:101920008A150E303702031D882CC33096005030C4
:101930009500CF2CB70137088A11A9218A15B70A5B
:10194000EB008A11E4228A150E303702031D9B2C0E
:10195000B5309000F430960024309500CF2CB701BC
:1019600037088A11BC218A15B70AEB008A11E422D4
:101970008A150E303702031DB02C83160C1100306F
:10198000F800043883129200093083169200831203
:1019900007110C309700960105309500CF2C2008D8
:1019A000023C0319D42CCF2C061BE82C831601080B
:1019B000C0390738810087308312900010108316D9
:1019C0000C1183122715270883168700142D831204
:1019D000861B122D36080D3C031DF02CB601F12C90
:1019E000B60A093003178D008F0103133608031759
:1019F0008C0083168C130C15831203130B08F7004D
:101A00008B138316031755308D00AA308D008C146C
:101A10008C18082D0C117708831203138B048A117C
:101A20002D268A15632B831683128A110A162B2FF3
:101A30000A148A100A1582076C2B892BA62BC32B3C
:101A4000E02BFD2B1A2C3B2C4E2C612C742C872C5C
:041A50009A2CAF2CF1
:1020000084011F308305073083169F00FF30831241
:10201000A700831681130108C03907388100873073
:10202000831290001010271227088316870083124E
:102030000712A71327088316870083128713A71296
:102040002708831687008312871227132708831611
:1020500087008312071327152708831687000614A5
:1020600086148312A710270883168700831287100F
:10207000A711270883168700831287110A128A2A5C
:102080000A16F0014030F1000A1274220A160230DA
:10209000EC000A1247220A160330B6008030B8005E
:1020A0000A12C5220A16B60B4E28B70137080A12C3
:1020B000CF210A16B70AB8000A12C5220A1605303F
:1020C0003702031D5628F0010330F1000A12742272
:1020D0000A160230EC000A1247220A16F0014830B4
:1020E000F1000A1274220A160230EC000A1247228A
:1020F0000A160E30B8000A12C5220A160A30B800B5
:102100000A12C5220A160E30B8000A12C5220A1693
:102110000530B6008030B8000A12C5220A16B60B88
:102120008A28F0010330F1000A1274220A160230E4
:10213000EC000A1247220A160A12CB220A1683164C
:102140000C1483128B15C0308B04B60136080A12AA
:1021500055200A1600380319B328B60AEB000A12F4
:10216000E4220A16A628B60136080A12D9210A1650
:10217000B60AEB000A12E4220A160D303602031DDD
:10218000B4280130EC000230ED000A12D3220A1606
:10219000B60136080A12EB210A16B60AEB000A123B
:1021A000E4220A160F303602031DC9280830B60093
:1021B000FA30EC000A1247220A16B60BD8280A1287
:1021C000B0230A167A08AB007908AA007808A9009B
:1021D0007708A8003510A001083003178D008F0183
:1021E00083168C130C1483120C080313B4003408E8
:1021F000FC3E0318302F043E582F3518E929BA0148
:102200003A080A1255200A16003803190D29BA0A8D
:10221000EB000A12E4220A160029BA013A080A124F
:102220005B200A16BA0AEB000A12E4220A160D30E5
:102230003A02031D0E290A12CB220A160830BA00F0
:10224000FA30EC000A1247220A16BA0B20290A12A9
:1022500005240A160830BA00FA30EC000A124722A8
:102260000A16BA0B2C290A12B0230A167A08B900EA
:102270007908B8007808B7007708B600E001DF01F8
:102280007930DE008830DD003908E4003808E300EA
:102290003708E2003608E1000A1239230A167708E7
:1022A000BA007808BB007908BC007A08BD000314A6
:1022B0002B08DC002A08DB002908DA002808D900EE
:1022C0003908E0003808DF003708DE003608DD0096
:1022D0000A120D240A163D08DB003C08DA003B0810
:1022E000D9003A08D8007A08DF007908DE007808BB
:1022F000DD007708DC000A124E250A167A08AF00C6
:102300007908AE007808AD007708AC00E630E00050
:10231000E930DF001D30DE008430DD002B08E400F2
:102320002A08E3002908E2002808E1000A123923FC
:102330000A167708BA007808BB007908BC007A084A
:10234000BD00E0007908DF007808DE007708DD00D6
:102350002F08E4002E08E3002D08E2002C08E1001D
:102360000A1239230A167708BE007808BF007908D8
:10237000C0007A08C100E0007908DF007808DE00BC
:102380007708DD00CC30E400BC30E3000C30E20024
:102390005730E1000A1239230A162830DB006B306F
:1023A000DA006E30D9009C30D8007A08DF00790856
:1023B000DE007808DD007708DC000A124E250A16D8
:1023C0007A08B3007908B2007808B1007708B00045
:1023D00035140A12CB220A160130EC000230ED004F
:1023E0000A12D3220A16B60136080A12FF210A166B
:1023F000B60AEB000A12E4220A1604303602031D64
:10240000F4290330B7002030EB000A12E4220A1648
:10241000B70B032A4330EB000A12E4220A16783085
:10242000EB000A12E4220A160330B8002030EB0059
:102430000A12E4220A16B80B162A0630B900390827
:102440000A12FF210A16B90AEB000A12E4220A1640
:102450000A303902031D1F2AC8013E30C700470851
:10246000413C031C442A470884004808C80ACA00A3
:1024700003178D008F0183168C130C1483120C0824
:1024800080000313C70A2F2A0A12B0230A167A08FB
:10249000B9007908B8007808B7007708B600200BB3
:1024A000522AA92A061B552AEE2B861BA82A3D086C
:1024B000C1003C08C0003B08BF003A08BE00C8018C
:1024C0003E30C7004708413C031C8D2A4808C80A13
:1024D000C900470884000008CA00490803178D0096
:1024E0008F0103134A0803178C0083168C130C15F5
:1024F000831203130B08F7008B1383160317553051
:102500008D00AA308D008C148C18842A0C11770849
:10251000831203138B04C70A622A0A121A260A16A8
:102520000630EC000130ED000A12D3220A16C90170
:1025300049080A1288200A16C90AEB000A12E42286
:102540000A1608304902031D982A0A122D260A1677
:10255000ED2B3908E1003808E0003708DF003608C5
:10256000DE00E501E4014830E3008530E2000A12B4
:1025700037260A16031CD72A0A121A260A16C90178
:1025800049080A1295200A16C90AEB000A12E42229
:102590000A160B304902031DC02A0330CA0021303D
:1025A000EB000A12E4220A16CA0BCF2AED2B2B08E5
:1025B000DB002A08DA002908D9002808D8003908E1
:1025C000DF003808DE003708DD003608DC000A12BC
:1025D0004E250A167708C9007808CA007908CB008A
:1025E0007A08CC0003147A08DC007908DB0078084C
:1025F000DA007708D900E001DF01DE017F30DD007D
:102600000A120D240A167708CD007808CE00790842
:10261000CF007A08D000E0007908DF007808DE00FB
:102620007708DD002F08E4002E08E3002D08E20003
:102630002C08E1000A1239230A167A08BD0079082D
:10264000BC007808BB007708BA0003143D08DC0022
:102650003C08DB003B08DA003A08D9004108E000FA
:102660004008DF003F08DE003E08DD000A120D24AE
:102670000A167A08C5007908C4007808C3007708EC
:10268000C2000A121A260A16D5014208F7004308AA
:10269000F8004408F9004508FA00F8134208D6008B
:1026A0007808D7004408D8004508D900E101E001C6
:1026B0007A30DF008830DE004508E5004408E40099
:1026C0007808E3004208E2000A1237260A16031CC3
:1026D000862B4508E0004408DF004308DE0042087E
:1026E000DD006F30E4001230E3000330E2007530AB
:1026F000E1000A1239230A167A08C5007908C400D5
:102700007808C3007708C200D50A452B5508F800A1
:102710007808C6004508D8004408D7004308D6000A
:102720004208D5000A1276260A167808063CC90027
:10273000EC000130ED000A12D3220A16E101E0019B
:10274000DF01DE014508E5004408E4004308E3003A
:102750004208E2000A1237260A160318B12B031D9D
:10276000B62B2030EB000A12E4220A16C608031D1D
:10277000C92B023084004508D9004408D80043081A
:10278000D7004208D6000A128A1500200A168A11BC
:10279000D82B033084004508D9004408D8004308EA
:1027A000D7004208D6000A128A1500200A168A119C
:1027B0000C30EC000130ED000A12D3220A16460854
:1027C0000A123D200A16C900EB000A12E4220A167A
:1027D0004630EB000A12E4220A16442AB401302FD4
:1027E0003518DC2CBA013A080A1255200A160038AE
:1027F0000319002CBA0AEB000A12E4220A16F32B82
:10280000BA013A080A125B200A16BA0AEB000A1249
:10281000E4220A160D303A02031D012C0A12CB22C3
:102820000A160830BA00FA30EC000A1247220A16DB
:10283000BA0B132C0A1205240A160830BA00FA3013
:10284000EC000A1247220A16BA0B1F2C0A12B023F8
:102850000A167A08B9007908B8007808B70077082E
:10286000B600E001DF017930DE008830DD00390894
:10287000E4003808E3003708E2003608E1000A12F5
:1028800039230A167708BA007808BB007908BC001B
:102890007A08BD0003142B08DC002A08DB00290895
:1028A000DA002808D9003908E0003808DF003708C6
:1028B000DE003608DD000A120D240A163D08DB0092
:1028C0003C08DA003B08D9003A08D8007A08DF0053
:1028D0007908DE007808DD007708DC000A124E2552
:1028E0000A167A08AF007908AE007808AD007708BC
:1028F000AC00E630E000E930DF001D30DE0084305F
:10290000DD002B08E4002A08E3002908E20028087B
:10291000E1000A1239230A167708BA007808BB00CA
:102920007908BC007A08BD00E0007908DF0078086B
:10293000DE007708DD002F08E4002E08E3002D08F4
:10294000E2002C08E1000A1239230A167708BE00BB
:102950007808BF007908C0007A08C100E000790853
:10296000DF007808DE007708DD00CC30E400BC3002
:10297000E3000C30E2005730E1000A1239230A1656
:102980002830DB006B30DA006E30D9009C30D80084
:102990007A08DF007908DE007808DD007708DC00BF
:1029A0000A124E250A167A08B3007908B200780890
:1029B000B1007708B00035140A12B82E0A1601309B
:1029C000EC000230ED000A12D3220A16B6013608D6
:1029D0000A120E220A16B60AEB000A12E4220A169E
:1029E00004303602031DE72C0330B7002030EB0023
:1029F0000A12E4220A16B70BF62C4C30EB000A122E
:102A0000E4220A167830EB000A12E4220A16033098
:102A1000B8002030EB000A12E4220A16B80B092D88
:102A20000630B90039080A120E220A16B90AEB005C
:102A30000A12E4220A160A303902031D122D04304C
:102A4000C8003E30C7004708413C031C382D4708EA
:102A500084004808C80ACA0003178D008F01831636
:102A60008C130C1483120C0880000313C70A232D47
:102A70000A12B0230A167A08B9007908B800780853
:102A8000B7007708B600200B462D9E2D061B492D5A
:102A9000EC2E861B9D2D3D08C1003C08C0003B0864
:102AA000BF003A08BE000430C8003E30C7004708E7
:102AB000413C031C822D4808C80AC900470884000D
:102AC0000008CA00490803178D008F0103134A0844
:102AD00003178C0083168C130C15831203130B0839
:102AE000F7008B138316031755308D00AA308D0025
:102AF0008C148C18792D0C117708831203138B0416
:102B0000C70A572D0A121A260A160930EC0001309E
:102B1000ED000A12D3220A16C90149080A126D20D3
:102B20000A16C90AEB000A12E4220A160530490205
:102B3000031D8D2D0A122D260A16EB2E3908E100F1
:102B40003808E0003708DF003608DE00E501E40160
:102B50004830E3008530E2000A1237260A16031CCB
:102B6000CC2D0A121A260A16C90149080A12772022
:102B70000A16C90AEB000A12E4220A160C304902AE
:102B8000031DB52D0330CA002130EB000A12E422E8
:102B90000A16CA0BC42DEB2E2B08DB002A08DA001C
:102BA0002908D9002808D8003908DF003808DE00D5
:102BB0003708DD003608DC000A124E250A167708B1
:102BC000C9007808CA007908CB007A08CC00031441
:102BD0007A08DC007908DB007808DA007708D90089
:102BE000E001DF01DE017F30DD000A120D240A164C
:102BF0007708CD007808CE007908CF007A08D00099
:102C0000E0007908DF007808DE007708DD0033088F
:102C1000E4003208E3003108E2003008E1000A1263
:102C200039230A167A08BD007908BC007808BB0071
:102C30007708BA0003143D08DC003C08DB003B08C1
:102C4000DA003A08D9004108E0004008DF003F08F8
:102C5000DE003E08DD000A120D240A167A08C500BF
:102C60007908C4007808C3007708C2000A121A263F
:102C70000A16D5014208F7004308F8004408F90095
:102C80004508FA00F8134208D6007808D70044082F
:102C9000D8004508D900E101E0017A30DF00883032
:102CA000DE004508E5004408E4007808E300420837
:102CB000E2000A1237260A16031C7B2E4508E000A4
:102CC0004408DF004308DE004208DD006F30E40006
:102CD0001230E3000330E2007530E1000A123923BC
:102CE0000A167A08C5007908C4007808C300770876
:102CF000C200D50A3A2E5508F8007808C6004508E3
:102D0000D8004408D7004308D6004208D5000A126C
:102D100076260A167808063CC900EC000130ED0062
:102D20000A12D3220A16E101E001DF01DE014508A3
:102D3000E5004408E4004308E3004208E2000A1208
:102D400037260A160318A62E031DAB2E2030EB00E3
:102D50000A12E4220A16C608031DC72E0330C90052
:102D60002030EB000A12E4220A16C90BB02E003004
:102D700084004508D9004408D8004308D700420819
:102D8000D6000A128A1500200A168A11D62E0330A0
:102D900084004508D9004408D8004308D7004208F9
:102DA000D6000A128A1500200A168A110C30EC008F
:102DB0000130ED000A12D3220A1646080A124520F5
:102DC0000A16C900EB000A12E4220A164830EB008A
:102DD0000A12E4220A16382D0230B400302F0A12EB
:102DE00005240A160130EC000230ED000A12D3224D
:102DF0000A16B60136080A121D220A16B60AEB0098
:102E00000A12E4220A1610303602031DFA2E1010A0
:102E10000A128A155B290A168A110330B400302F72
:102E20000A1205240A160130EC000230ED000A12E5
:102E3000D3220A16B60136080A1232220A16B60A38
:102E4000EB000A12E4220A1610303602031D1B2F73
:102E50000A128A154B2B0A168A110130B400302F42
:102E6000083003178D008F010313340803178C00FB
:102E700083168C130C15831203130B08F7008B13A6
:102E80008316031755308D00AA308D008C148C18D2
:102E9000472F0C117708831203138B040A122D2677
:102EA0000A160A30EC000A1247220A16F7286300B5
:102EB0000A148A140A158207F02BFD28EF2E102F12
:1042000000000000000000000000000000000000AE
:0442100001000D009C
:02400E00393F38
:00000001FF
